 wavedev2_sgtl5000

 Timestamp is 4fb04cbb (Mon May 14 12:07:23 2012)

 Preferred load address is 10000000

 Start         Length     Name                   Class
 0001:00000000 00000004H .CRT$XCA                CODE
 0001:00000004 00000004H .CRT$XCZ                CODE
 0001:00000008 00000004H .CRT$XIA                CODE
 0001:0000000c 00000004H .CRT$XIZ                CODE
 0001:00000010 00000004H .CRT$XPA                CODE
 0001:00000014 00000004H .CRT$XPZ                CODE
 0001:00000018 00000004H .CRT$XTA                CODE
 0001:0000001c 00000004H .CRT$XTZ                CODE
 0001:00000020 00000b0aH .rdata                  CODE
 0001:00000b2c 0000002eH .rdata$debug            CODE
 0001:00000b5c 00008910H .text                   CODE
 0001:0000946c 00000064H .xdata                  CODE
 0001:000094d0 00000064H .idata$2                CODE
 0001:00009534 00000014H .idata$3                CODE
 0001:00009548 00000128H .idata$4                CODE
 0001:00009670 00000196H .idata$6                CODE
 0001:00009810 000000a1H .edata                  CODE
 0002:00000000 00000128H .idata$5                DATA
 0002:00000128 000000c0H .data                   DATA
 0002:000001e8 00000068H .bss                    DATA
 0003:00000000 00000930H .pdata                  DATA

  Address         Publics by Value              Rva+Base       Lib:Object

 0000:00000000       ___safe_se_handler_count   00000000     <absolute>
 0000:00000000       ___safe_se_handler_table   00000000     <absolute>
 0001:00000000       __xc_a                     10001000     corelib0:crt0init.obj
 0001:00000004       __xc_z                     10001004     corelib0:crt0init.obj
 0001:00000008       __xi_a                     10001008     corelib0:crt0init.obj
 0001:0000000c       __xi_z                     1000100c     corelib0:crt0init.obj
 0001:00000010       __xp_a                     10001010     corelib0:crt0init.obj
 0001:00000014       __xp_z                     10001014     corelib0:crt0init.obj
 0001:00000018       __xt_a                     10001018     corelib0:crt0init.obj
 0001:0000001c       __xt_z                     1000101c     corelib0:crt0init.obj
 0001:0000003c       ??_C@_1M@LCEEOPDH@?$AAI?$AA2?$AAC?$AA1?$AA?3?$AA?$AA@ 1000103c     sgtl5000codec.obj
 0001:00000048       ??_7InputDeviceContext@@6B@ 10001048     wavedev2_common_topaz_v1:hwctxt.obj
 0001:00000068       ??_7OutputDeviceContext@@6B@ 10001068     wavedev2_common_topaz_v1:hwctxt.obj
 0001:00000088       ??_C@_1BI@BHLBGEOK@?$AAP?$AAr?$AAi?$AAo?$AAr?$AAi?$AAt?$AAy?$AA2?$AA5?$AA6?$AA?$AA@ 10001088     wavedev2_common_topaz_v1:hwctxt.obj
 0001:000000a0       ??_7DeviceContext@@6B@     100010a0     wavedev2_common_topaz_v1:devctxt.obj
 0001:000000dc       ??_7CMidiStream@@6B@       100010dc     wavedev2_common_topaz_v1:devctxt.obj
 0001:00000128       ??_7InputStreamContext@@6B@ 10001128     wavedev2_common_topaz_v1:devctxt.obj
 0001:00000170       ??_7OutputStreamContext16bitM8@@6B@ 10001170     wavedev2_common_topaz_v1:devctxt.obj
 0001:000001b8       ??_7OutputStreamContext16bitS8@@6B@ 100011b8     wavedev2_common_topaz_v1:devctxt.obj
 0001:00000200       ??_7OutputStreamContext16bitM16@@6B@ 10001200     wavedev2_common_topaz_v1:devctxt.obj
 0001:00000248       ??_7OutputStreamContext16bitS16@@6B@ 10001248     wavedev2_common_topaz_v1:devctxt.obj
 0001:00000290       ??_7OutputStreamContext24bitM8@@6B@ 10001290     wavedev2_common_topaz_v1:devctxt.obj
 0001:000002d8       ??_7OutputStreamContext24bitS8@@6B@ 100012d8     wavedev2_common_topaz_v1:devctxt.obj
 0001:00000320       ??_7OutputStreamContext24bitM16@@6B@ 10001320     wavedev2_common_topaz_v1:devctxt.obj
 0001:00000368       ??_7OutputStreamContext24bitS16@@6B@ 10001368     wavedev2_common_topaz_v1:devctxt.obj
 0001:000003b0       ??_7OutputStreamContext24bitS24@@6B@ 100013b0     wavedev2_common_topaz_v1:devctxt.obj
 0001:00000588       ??_7StreamContext@@6B@     10001588     wavedev2_common_topaz_v1:strmctxt.obj
 0001:000005c4       ??_C@_1BC@JBIMOOCB@?$AAP?$AAl?$AAa?$AAy?$AAb?$AAa?$AAc?$AAk?$AA?$AA@ 100015c4     wavedev2_common_topaz_v1:mixerdrv.obj
 0001:000005d8       ??_C@_1BA@EEOGCIBB@?$AAL?$AAi?$AAn?$AAe?$AA?5?$AAI?$AAn?$AA?$AA@ 100015d8     wavedev2_common_topaz_v1:mixerdrv.obj
 0001:000005e8       ??_C@_1BG@OGJPAHBK@?$AAM?$AAi?$AAc?$AAr?$AAo?$AAp?$AAh?$AAo?$AAn?$AAe?$AA?$AA@ 100015e8     wavedev2_common_topaz_v1:mixerdrv.obj
 0001:00000600       ??_C@_1CE@BJPEGCKG@?$AAR?$AAe?$AAc?$AAo?$AAr?$AAd?$AAi?$AAn?$AAg?$AA?5?$AAC?$AAo?$AAn?$AAt?$AAr?$AAo?$AAl?$AA?$AA@ 10001600     wavedev2_common_topaz_v1:mixerdrv.obj
 0001:00000624       ??_C@_1CA@KOFAABPH@?$AAR?$AAe?$AAc?$AAo?$AAr?$AAd?$AAi?$AAn?$AAg?$AA?5?$AAC?$AAo?$AAn?$AAt?$AAr?$AA?$AA@ 10001624     wavedev2_common_topaz_v1:mixerdrv.obj
 0001:00000644       ??_C@_1CC@OALPFLIM@?$AAP?$AAl?$AAa?$AAy?$AAb?$AAa?$AAc?$AAk?$AA?5?$AAC?$AAo?$AAn?$AAt?$AAr?$AAo?$AAl?$AA?$AA@ 10001644     wavedev2_common_topaz_v1:mixerdrv.obj
 0001:00000668       ??_C@_1BO@OJJBHHKI@?$AAP?$AAl?$AAa?$AAy?$AAb?$AAa?$AAc?$AAk?$AA?5?$AAC?$AAo?$AAn?$AAt?$AAr?$AA?$AA@ 10001668     wavedev2_common_topaz_v1:mixerdrv.obj
 0001:00000744       ??_7MixerControl@@6B@      10001744     wavedev2_common_topaz_v1:mixerdrv.obj
 0001:00000760       ??_7MixerControlVolumeMaster@@6B@ 10001760     wavedev2_common_topaz_v1:mixerdrv.obj
 0001:00000784       ??_C@_1BM@DBCMFCBE@?$AAM?$AAa?$AAs?$AAt?$AAe?$AAr?$AA?5?$AAV?$AAo?$AAl?$AAu?$AAm?$AAe?$AA?$AA@ 10001784     wavedev2_common_topaz_v1:mixerdrv.obj
 0001:000007a0       ??_7MixerControlVolumeMic@@6B@ 100017a0     wavedev2_common_topaz_v1:mixerdrv.obj
 0001:000007c4       ??_C@_1BG@LAGONMFD@?$AAM?$AAi?$AAc?$AA?5?$AAV?$AAo?$AAl?$AAu?$AAm?$AAe?$AA?$AA@ 100017c4     wavedev2_common_topaz_v1:mixerdrv.obj
 0001:000007dc       ??_7MixerControlMuteMaster@@6B@ 100017dc     wavedev2_common_topaz_v1:mixerdrv.obj
 0001:00000800       ??_C@_1BI@PEAJCPFH@?$AAM?$AAa?$AAs?$AAt?$AAe?$AAr?$AA?5?$AAM?$AAu?$AAt?$AAe?$AA?$AA@ 10001800     wavedev2_common_topaz_v1:mixerdrv.obj
 0001:00000818       ??_7MixerControlMuteMic@@6B@ 10001818     wavedev2_common_topaz_v1:mixerdrv.obj
 0001:0000083c       ??_C@_1BC@MOMKCGGI@?$AAM?$AAi?$AAc?$AA?5?$AAM?$AAu?$AAt?$AAe?$AA?$AA@ 1000183c     wavedev2_common_topaz_v1:mixerdrv.obj
 0001:00000850       ??_7MixerControlLoopback@@6B@ 10001850     wavedev2_common_topaz_v1:mixerdrv.obj
 0001:00000874       ??_C@_1CC@NMFCMAHN@?$AAL?$AAo?$AAo?$AAp?$AAb?$AAa?$AAc?$AAk?$AA?5?$AAC?$AAo?$AAn?$AAt?$AAr?$AAo?$AAl?$AA?$AA@ 10001874     wavedev2_common_topaz_v1:mixerdrv.obj
 0001:00000898       ??_C@_1BC@NMCMBANA@?$AAL?$AAo?$AAo?$AAp?$AAb?$AAa?$AAc?$AAk?$AA?$AA@ 10001898     wavedev2_common_topaz_v1:mixerdrv.obj
 0001:000008ac       ??_7MixerControlInputMux@@6B@ 100018ac     wavedev2_common_topaz_v1:mixerdrv.obj
 0001:000008c8       ??_7MixerControlList@@6B@  100018c8     wavedev2_common_topaz_v1:mixerdrv.obj
 0001:000008cc       ??_C@_1BI@DKACBKCL@?$AAA?$AAu?$AAd?$AAi?$AAo?$AA?5?$AAM?$AAi?$AAx?$AAe?$AAr?$AA?$AA@ 100018cc     wavedev2_common_topaz_v1:mixerdrv.obj
 0001:000008e4       ??_C@_1BE@FNMPOHBO@?$AAI?$AAn?$AAp?$AAu?$AAt?$AA?5?$AAM?$AAu?$AAx?$AA?$AA@ 100018e4     wavedev2_common_topaz_v1:mixerdrv.obj
 0001:000008f8       ?ms_BasePitchTable@CMidiStream@@0QBKB 100018f8     wavedev2_common_topaz_v1:midistrm.obj
 0001:00000928       ?SineTable@CMidiNote@@0QBFB 10001928     wavedev2_common_topaz_v1:midinote.obj
 0001:00000b5c       ?BSPAudioStartDAC@@YAXXZ   10001b5c f   bsphwctxt.obj
 0001:00000b7c       ?BSPAudioStopDAC@@YAXXZ    10001b7c f   bsphwctxt.obj
 0001:00000b9c       ?BSPAudioStartADC@@YAXXZ   10001b9c f   bsphwctxt.obj
 0001:00000bbc       ?BSPAudioStopADC@@YAXXZ    10001bbc f   bsphwctxt.obj
 0001:00000bdc       ?BSPSetSpeakerEnable@@YAXH@Z 10001bdc f   bsphwctxt.obj
 0001:00000c0c       ?BSPAudioSelectADCSource@@YAXK@Z 10001c0c f   bsphwctxt.obj
 0001:00000c34       ?BSPAudioSetCodecLoopback@@YAHH@Z 10001c34 f   bsphwctxt.obj
 0001:00000c3c       ?BSPAudioSetOutputGain@@YAXK@Z 10001c3c f   bsphwctxt.obj
 0001:00000d64       ?BSPAudioSetInputGain@@YAXK@Z 10001d64 f   bsphwctxt.obj
 0001:00000d90       ?BSPAudioGetInputDeviceNum@@YAEXZ 10001d90 f   bsphwctxt.obj
 0001:00000d98       ?BSPAllocOutputDMABuffer@@YAGPAPAEPAT_LARGE_INTEGER@@@Z 10001d98 f   bsphwctxt.obj
 0001:00000dd8       ?BSPDeallocOutputDMABuffer@@YAXPAE@Z 10001dd8 f   bsphwctxt.obj
 0001:00000ddc       ?BSPAllocInputDMABuffer@@YAGPAPAEPAT_LARGE_INTEGER@@@Z 10001ddc f   bsphwctxt.obj
 0001:00000e30       ?BSPDeallocInputDMABuffer@@YAXPAE@Z 10001e30 f   bsphwctxt.obj
 0001:00000e88       ?BSPAudioIomuxConfig@@YAXXZ 10001e88 f   bsphwctxt.obj
 0001:00000ed4       ?BSPSsiEnableClock@@YAHIH@Z 10001ed4 f   bsphwctxt.obj
 0001:00000f14       ?BSPAudmuxEnableClock@@YAHH@Z 10001f14 f   bsphwctxt.obj
 0001:00000f34       ?BSPGetAudmuxIntPort@@YA?AW4AUDMUX_INTERNAL_PORT@@XZ 10001f34 f   bsphwctxt.obj
 0001:00000f3c       ?BSPGetAudmuxExtPort@@YA?AW4AUDMUX_EXTERNAL_PORT@@XZ 10001f3c f   bsphwctxt.obj
 0001:00000f44       ?BSPAudioGetSdmaPriority@@YAEXZ 10001f44 f   bsphwctxt.obj
 0001:00000f4c       ?BSPAudioPowerUp@@YAXH@Z   10001f4c f   bsphwctxt.obj
 0001:00000f70       ?BSPAudioPowerDown@@YAXH@Z 10001f70 f   bsphwctxt.obj
 0001:00000f94       ?BSPAudioGetProtocol@@YA?AW4AUDIO_PROTOCOL@@XZ 10001f94 f   bsphwctxt.obj
 0001:00000f9c       ?BSPIsHeadphoneDetectSupported@@YAHXZ 10001f9c f   bsphwctxt.obj
 0001:00000fa4       ?BSPGetHPDetectIRQ@@YAKXZ  10001fa4 f   bsphwctxt.obj
 0001:00000fac       ?BSPAudioHandleHPDetectIRQ@@YAXXZ 10001fac f   bsphwctxt.obj
 0001:00000fb0       ?BSPGetBitsPerSample@@YAGXZ 10001fb0 f   bsphwctxt.obj
 0001:00000fb8       ?BSPAudioDeinitCodec@@YAXXZ 10001fb8 f   bsphwctxt.obj
 0001:00000ffc       ?BSPAudioInitCodec@@YAHXZ  10001ffc f   bsphwctxt.obj
 0001:00001070       ?SGTL5000I2CClose@SGTL5000Codec@@QAAXXZ 10002070 f   sgtl5000codec.obj
 0001:000010ac       ?SGTL5000WriteRegister@SGTL5000Codec@@QAAIGG@Z 100020ac f   sgtl5000codec.obj
 0001:00001130       ?SGTL5000ReadRegister@SGTL5000Codec@@QAAIGPAG@Z 10002130 f   sgtl5000codec.obj
 0001:000011e0       ?SGTL5000ModifyRegister@SGTL5000Codec@@QAAIGGG@Z 100021e0 f   sgtl5000codec.obj
 0001:00001248       ?SGTL5000ConfigureDuplexMode@SGTL5000Codec@@QAAXXZ 10002248 f   sgtl5000codec.obj
 0001:00001294       ?SGTL5000RampHPVolume@SGTL5000Codec@@QAAXG@Z 10002294 f   sgtl5000codec.obj
 0001:00001344       ?SGTL5000SetDACVolume@SGTL5000Codec@@QAAXEE@Z 10002344 f   sgtl5000codec.obj
 0001:00001364       ?SGTL5000SetADCVolume@SGTL5000Codec@@QAAXEE@Z 10002364 f   sgtl5000codec.obj
 0001:00001388       ?SGTL5000SetADCInput@SGTL5000Codec@@QAAXW4SGTL5000_ADC_INPUT@@@Z 10002388 f   sgtl5000codec.obj
 0001:000013b8       ?SGTL5000ForceSpeaker@SGTL5000Codec@@QAAXI@Z 100023b8 f   sgtl5000codec.obj
 0001:000013c0       ?SGTL5000SpeakerHeadphoneSelection@SGTL5000Codec@@QAAXXZ 100023c0 f   sgtl5000codec.obj
 0001:00001428       ??1SGTL5000Codec@@QAA@XZ   10002428 f   sgtl5000codec.obj
 0001:00001440       ?SGTL5000I2CInit@SGTL5000Codec@@QAAIXZ 10002440 f   sgtl5000codec.obj
 0001:000014c8       ?SGTL5000CodecInit@SGTL5000Codec@@QAAIXZ 100024c8 f   sgtl5000codec.obj
 0001:00001598       ?SGTL5000ConfigureLoopbackMode@SGTL5000Codec@@QAAXXZ 10002598 f   sgtl5000codec.obj
 0001:00001640       ?SGTL5000ConfigurePowerMode@SGTL5000Codec@@QAAXG@Z 10002640 f   sgtl5000codec.obj
 0001:0000196c       ??0SGTL5000Codec@@QAA@XZ   1000296c f   sgtl5000codec.obj
 0001:000019a0       DllMain                    100029a0 f   wavedev2_common_topaz_v1:wavemain.obj
 0001:000019b8       WAV_Init                   100029b8 f   wavedev2_common_topaz_v1:wavemain.obj
 0001:000019c8       WAV_Deinit                 100029c8 f   wavedev2_common_topaz_v1:wavemain.obj
 0001:000019e4       WAV_Open                   100029e4 f   wavedev2_common_topaz_v1:wavemain.obj
 0001:00001a0c       WAV_Close                  10002a0c f   wavedev2_common_topaz_v1:wavemain.obj
 0001:00001a28       ?HandleWaveMessage@@YAHPAUMMDRV_MESSAGE_PARAMS@@PAK@Z 10002a28 f   wavedev2_common_topaz_v1:wavemain.obj
 0001:00001ee0       WAV_IOControl              10002ee0 f   wavedev2_common_topaz_v1:wavemain.obj
 0001:00001fe4       ?Deinit@HardwareContext@@QAAHXZ 10002fe4 f   wavedev2_common_topaz_v1:hwctxt.obj
 0001:000020dc       ?InitSsi@HardwareContext@@AAAXW4AUDIO_PROTOCOL@@@Z 100030dc f   wavedev2_common_topaz_v1:hwctxt.obj
 0001:00002214       ?InitAudmux@HardwareContext@@AAAXW4AUDMUX_INTERNAL_PORT@@W4AUDMUX_EXTERNAL_PORT@@@Z 10003214 f   wavedev2_common_topaz_v1:hwctxt.obj
 0001:0000227c       ?InitOutputDMA@HardwareContext@@AAAHXZ 1000327c f   wavedev2_common_topaz_v1:hwctxt.obj
 0001:000023e4       ?InitInputDMA@HardwareContext@@AAAHXZ 100033e4 f   wavedev2_common_topaz_v1:hwctxt.obj
 0001:0000256c       ?StopCodec@HardwareContext@@AAAXW4AUDIO_BUS@@@Z 1000356c f   wavedev2_common_topaz_v1:hwctxt.obj
 0001:00002624       ?StartSsi@HardwareContext@@AAAXW4AUDIO_BUS@@@Z 10003624 f   wavedev2_common_topaz_v1:hwctxt.obj
 0001:00002734       ?StopSsi@HardwareContext@@AAAXW4AUDIO_BUS@@@Z 10003734 f   wavedev2_common_topaz_v1:hwctxt.obj
 0001:00002840       ?StopOutputDMA@HardwareContext@@QAAXXZ 10003840 f   wavedev2_common_topaz_v1:hwctxt.obj
 0001:000028a0       ?StartInputDMA@HardwareContext@@QAAHXZ 100038a0 f   wavedev2_common_topaz_v1:hwctxt.obj
 0001:00002998       ?StopInputDMA@HardwareContext@@QAAXXZ 10003998 f   wavedev2_common_topaz_v1:hwctxt.obj
 0001:000029f8       ?TransferBuffer@HardwareContext@@IAAKW4AUDIO_BUS@@E@Z 100039f8 f   wavedev2_common_topaz_v1:hwctxt.obj
 0001:00002a88       ?HPDetectInterruptThread@HardwareContext@@QAAXXZ 10003a88 f   wavedev2_common_topaz_v1:hwctxt.obj
 0001:00002af4       ?DisableDelayThread@HardwareContext@@QAAXXZ 10003af4 f   wavedev2_common_topaz_v1:hwctxt.obj
 0001:00002c00       ?CallDisableDelayThread@@YAXPAVHardwareContext@@@Z 10003c00 f   wavedev2_common_topaz_v1:hwctxt.obj
 0001:00002c10       ?CallHPDetectInterruptThread@@YAXPAVHardwareContext@@@Z 10003c10 f   wavedev2_common_topaz_v1:hwctxt.obj
 0001:00002c20       ?SetOutputGain@HardwareContext@@QAAIK@Z 10003c20 f   wavedev2_common_topaz_v1:hwctxt.obj
 0001:00002c48       ?SetOutputMute@HardwareContext@@QAAIH@Z 10003c48 f   wavedev2_common_topaz_v1:hwctxt.obj
 0001:00002c6c       ?GetOutputGain@HardwareContext@@QAAKXZ 10003c6c f   wavedev2_common_topaz_v1:hwctxt.obj
 0001:00002c74       ?GetOutputMute@HardwareContext@@QAAHXZ 10003c74 f   wavedev2_common_topaz_v1:hwctxt.obj
 0001:00002c7c       ?GetInputMute@HardwareContext@@QAAHXZ 10003c7c f   wavedev2_common_topaz_v1:hwctxt.obj
 0001:00002c84       ?SetInputMute@HardwareContext@@QAAIH@Z 10003c84 f   wavedev2_common_topaz_v1:hwctxt.obj
 0001:00002ca8       ?GetInputGain@HardwareContext@@QAAKXZ 10003ca8 f   wavedev2_common_topaz_v1:hwctxt.obj
 0001:00002cb0       ?SetInputGain@HardwareContext@@QAAIK@Z 10003cb0 f   wavedev2_common_topaz_v1:hwctxt.obj
 0001:00002cd8       ?ForceSpeaker@HardwareContext@@QAAKH@Z 10003cd8 f   wavedev2_common_topaz_v1:hwctxt.obj
 0001:00002d20       ?PowerDown@HardwareContext@@QAAXXZ 10003d20 f   wavedev2_common_topaz_v1:hwctxt.obj
 0001:00002db0       ?GetDriverRegValue@HardwareContext@@QAAKPAGK@Z 10003db0 f   wavedev2_common_topaz_v1:hwctxt.obj
 0001:00002e18       ?IsSupportedOutputFormat@HardwareContext@@QAAHPAUtWAVEFORMATEX@@@Z 10003e18 f   wavedev2_common_topaz_v1:hwctxt.obj
 0001:00002e20       ?SelectInputSource@HardwareContext@@QAAHK@Z 10003e20 f   wavedev2_common_topaz_v1:hwctxt.obj
 0001:00002e64       ?SetCodecLoopback@HardwareContext@@QAAHH@Z 10003e64 f   wavedev2_common_topaz_v1:hwctxt.obj
 0001:00002edc       ??0HardwareContext@@QAA@XZ 10003edc f   wavedev2_common_topaz_v1:hwctxt.obj
 0001:00002f38       ?InitHPDetectInterruptThread@HardwareContext@@IAAHXZ 10003f38 f   wavedev2_common_topaz_v1:hwctxt.obj
 0001:00002ffc       ?InitDisableDelayThread@HardwareContext@@IAAHXZ 10003ffc f   wavedev2_common_topaz_v1:hwctxt.obj
 0001:000030fc       ?TransferOutputBuffers@HardwareContext@@IAAKXZ 100040fc f   wavedev2_common_topaz_v1:hwctxt.obj
 0001:0000316c       ?TransferInputBuffers@HardwareContext@@IAAKE@Z 1000416c f   wavedev2_common_topaz_v1:hwctxt.obj
 0001:00003268       ?OutputIntrRoutine@HardwareContext@@AAAXXZ 10004268 f   wavedev2_common_topaz_v1:hwctxt.obj
 0001:00003374       ?InputIntrRoutine@HardwareContext@@AAAXXZ 10004374 f   wavedev2_common_topaz_v1:hwctxt.obj
 0001:000034d4       ?StartOutputDMA@HardwareContext@@QAAHXZ 100044d4 f   wavedev2_common_topaz_v1:hwctxt.obj
 0001:0000360c       ?InterruptThread@HardwareContext@@QAAXXZ 1000460c f   wavedev2_common_topaz_v1:hwctxt.obj
 0001:00003690       ?CallInterruptThread@@YAXPAVHardwareContext@@@Z 10004690 f   wavedev2_common_topaz_v1:hwctxt.obj
 0001:000036a0       ?PowerUp@HardwareContext@@QAAXXZ 100046a0 f   wavedev2_common_topaz_v1:hwctxt.obj
 0001:000036f8       ?InitInterruptThread@HardwareContext@@IAAHXZ 100046f8 f   wavedev2_common_topaz_v1:hwctxt.obj
 0001:000037a4       ?PmControlMessage@HardwareContext@@QAAHKPAEK0KPAK@Z 100047a4 f   wavedev2_common_topaz_v1:hwctxt.obj
 0001:000038d8       ?Init@HardwareContext@@QAAHK@Z 100048d8 f   wavedev2_common_topaz_v1:hwctxt.obj
 0001:00003a88       ?CreateHWContext@HardwareContext@@SAHK@Z 10004a88 f   wavedev2_common_topaz_v1:hwctxt.obj
 0001:00003aec       ??0DeviceContext@@QAA@XZ   10004aec f   wavedev2_common_topaz_v1:devctxt.obj
 0001:00003b3c       ?GetGain@DeviceContext@@QAAKXZ 10004b3c f   wavedev2_common_topaz_v1:devctxt.obj
 0001:00003b44       ?GetDefaultStreamGain@DeviceContext@@QAAKXZ 10004b44 f   wavedev2_common_topaz_v1:devctxt.obj
 0001:00003b4c       ?GetSecondaryGainLimit@DeviceContext@@QAAKK@Z 10004b4c f   wavedev2_common_topaz_v1:devctxt.obj
 0001:00003b58       ?IsSupportedFormat@DeviceContext@@UAAHPAUtWAVEFORMATEX@@@Z 10004b58 f   wavedev2_common_topaz_v1:devctxt.obj
 0001:00003c38       ?IsSupportedFormat@OutputDeviceContext@@UAAHPAUtWAVEFORMATEX@@@Z 10004c38 f   wavedev2_common_topaz_v1:devctxt.obj
 0001:00003c94       ?NewStream@DeviceContext@@UAAKPAVStreamContext@@@Z 10004c94 f   wavedev2_common_topaz_v1:devctxt.obj
 0001:00003d1c       ?DeleteStream@DeviceContext@@QAAXPAVStreamContext@@@Z 10004d1c f   wavedev2_common_topaz_v1:devctxt.obj
 0001:00003d68       ?TransferBuffer@DeviceContext@@QAAPAEPAE0PAUTRANSFER_STATUS@@@Z 10004d68 f   wavedev2_common_topaz_v1:devctxt.obj
 0001:00003e08       ?RecalcAllGains@DeviceContext@@QAAXXZ 10004e08 f   wavedev2_common_topaz_v1:devctxt.obj
 0001:00003e40       ?StreamReadyToRender@OutputDeviceContext@@UAAXPAVStreamContext@@@Z 10004e40 f   wavedev2_common_topaz_v1:devctxt.obj
 0001:00003e5c       ?StreamReadyToRender@InputDeviceContext@@UAAXPAVStreamContext@@@Z 10004e5c f   wavedev2_common_topaz_v1:devctxt.obj
 0001:00003e78       ?GetDevCaps@OutputDeviceContext@@UAAKPAXK@Z 10004e78 f   wavedev2_common_topaz_v1:devctxt.obj
 0001:00003ebc       ?GetDevCaps@InputDeviceContext@@UAAKPAXK@Z 10004ebc f   wavedev2_common_topaz_v1:devctxt.obj
 0001:00003f00       ?GetExtDevCaps@OutputDeviceContext@@UAAKPAXK@Z 10004f00 f   wavedev2_common_topaz_v1:devctxt.obj
 0001:00003f28       ?GetExtDevCaps@InputDeviceContext@@UAAKPAXK@Z 10004f28 f   wavedev2_common_topaz_v1:devctxt.obj
 0001:00003f30       ?OpenStream@DeviceContext@@QAAKPAUwaveopendesc_tag@@KPAPAVStreamContext@@@Z 10004f30 f   wavedev2_common_topaz_v1:devctxt.obj
 0001:00004008       ?ResetBaseInfo@DeviceContext@@QAAXXZ 10005008 f   wavedev2_common_topaz_v1:devctxt.obj
 0001:00004040       ?GetBaseSampleRate@DeviceContext@@QAAKXZ 10005040 f   wavedev2_common_topaz_v1:devctxt.obj
 0001:00004048       ?GetBaseSampleRateInverse@DeviceContext@@QAAKXZ 10005048 f   wavedev2_common_topaz_v1:devctxt.obj
 0001:00004050       ?GetChannels@OutputDeviceContext@@UAAKXZ 10005050 f   wavedev2_common_topaz_v1:devctxt.obj
 0001:00004058       ?GetChannels@InputDeviceContext@@UAAKXZ 10005058 f   wavedev2_common_topaz_v1:devctxt.obj
 0001:00004060       ?GetNativeFormat@DeviceContext@@QAAKKPAXKPAK@Z 10005060 f   wavedev2_common_topaz_v1:devctxt.obj
 0001:0000411c       ?GetProperty@DeviceContext@@QAAKPAUtag_WAVEPROPINFO@@@Z 1000511c f   wavedev2_common_topaz_v1:devctxt.obj
 0001:00004204       ?SetProperty@DeviceContext@@QAAKPAUtag_WAVEPROPINFO@@@Z 10005204 f   wavedev2_common_topaz_v1:devctxt.obj
 0001:0000420c       ?SetSecondaryGainLimit@DeviceContext@@QAAKKK@Z 1000520c f   wavedev2_common_topaz_v1:devctxt.obj
 0001:00004238       ??_EInputStreamContext@@UAAPAXI@Z 10005238 f i wavedev2_common_topaz_v1:devctxt.obj
 0001:00004238       ??_GInputStreamContext@@UAAPAXI@Z 10005238 f i wavedev2_common_topaz_v1:devctxt.obj
 0001:00004260       ??_ECMidiStream@@UAAPAXI@Z 10005260 f i wavedev2_common_topaz_v1:devctxt.obj
 0001:00004260       ??_GCMidiStream@@UAAPAXI@Z 10005260 f i wavedev2_common_topaz_v1:devctxt.obj
 0001:00004288       ??_GOutputStreamContext16bitM8@@UAAPAXI@Z 10005288 f i wavedev2_common_topaz_v1:devctxt.obj
 0001:00004288       ??_EOutputStreamContext16bitM8@@UAAPAXI@Z 10005288 f i wavedev2_common_topaz_v1:devctxt.obj
 0001:000042b0       ??_GOutputStreamContext16bitS8@@UAAPAXI@Z 100052b0 f i wavedev2_common_topaz_v1:devctxt.obj
 0001:000042b0       ??_EOutputStreamContext16bitS8@@UAAPAXI@Z 100052b0 f i wavedev2_common_topaz_v1:devctxt.obj
 0001:000042d8       ??_EOutputStreamContext16bitM16@@UAAPAXI@Z 100052d8 f i wavedev2_common_topaz_v1:devctxt.obj
 0001:000042d8       ??_GOutputStreamContext16bitM16@@UAAPAXI@Z 100052d8 f i wavedev2_common_topaz_v1:devctxt.obj
 0001:00004300       ??_EOutputStreamContext16bitS16@@UAAPAXI@Z 10005300 f i wavedev2_common_topaz_v1:devctxt.obj
 0001:00004300       ??_GOutputStreamContext16bitS16@@UAAPAXI@Z 10005300 f i wavedev2_common_topaz_v1:devctxt.obj
 0001:00004328       ??_GOutputStreamContext24bitM8@@UAAPAXI@Z 10005328 f i wavedev2_common_topaz_v1:devctxt.obj
 0001:00004328       ??_EOutputStreamContext24bitM8@@UAAPAXI@Z 10005328 f i wavedev2_common_topaz_v1:devctxt.obj
 0001:00004350       ??_EOutputStreamContext24bitS8@@UAAPAXI@Z 10005350 f i wavedev2_common_topaz_v1:devctxt.obj
 0001:00004350       ??_GOutputStreamContext24bitS8@@UAAPAXI@Z 10005350 f i wavedev2_common_topaz_v1:devctxt.obj
 0001:00004378       ??_EOutputStreamContext24bitM16@@UAAPAXI@Z 10005378 f i wavedev2_common_topaz_v1:devctxt.obj
 0001:00004378       ??_GOutputStreamContext24bitM16@@UAAPAXI@Z 10005378 f i wavedev2_common_topaz_v1:devctxt.obj
 0001:000043a0       ??_GOutputStreamContext24bitS16@@UAAPAXI@Z 100053a0 f i wavedev2_common_topaz_v1:devctxt.obj
 0001:000043a0       ??_EOutputStreamContext24bitS16@@UAAPAXI@Z 100053a0 f i wavedev2_common_topaz_v1:devctxt.obj
 0001:000043c8       ??_EOutputStreamContext24bitS24@@UAAPAXI@Z 100053c8 f i wavedev2_common_topaz_v1:devctxt.obj
 0001:000043c8       ??_GOutputStreamContext24bitS24@@UAAPAXI@Z 100053c8 f i wavedev2_common_topaz_v1:devctxt.obj
 0001:000043f0       ?SetBaseSampleRate@DeviceContext@@UAAXK@Z 100053f0 f   wavedev2_common_topaz_v1:devctxt.obj
 0001:0000442c       ?CreateStream@InputDeviceContext@@UAAPAVStreamContext@@PAUwaveopendesc_tag@@@Z 1000542c f   wavedev2_common_topaz_v1:devctxt.obj
 0001:00004468       ?CreateStream@OutputDeviceContext@@UAAPAVStreamContext@@PAUwaveopendesc_tag@@@Z 10005468 f   wavedev2_common_topaz_v1:devctxt.obj
 0001:00004728       ??0StreamContext@@QAA@XZ   10005728 f   wavedev2_common_topaz_v1:strmctxt.obj
 0001:0000473c       ??1StreamContext@@UAA@XZ   1000573c f   wavedev2_common_topaz_v1:strmctxt.obj
 0001:0000474c       ?StillPlaying@StreamContext@@QAAHXZ 1000574c f   wavedev2_common_topaz_v1:strmctxt.obj
 0001:00004760       ?GetDeviceContext@StreamContext@@QAAPAVDeviceContext@@XZ 10005760 f   wavedev2_common_topaz_v1:strmctxt.obj
 0001:00004768       ?DoDriverCallback@StreamContext@@QAAXIKK@Z 10005768 f   wavedev2_common_topaz_v1:strmctxt.obj
 0001:000047a0       ?DoCallbackReturnBuffer@StreamContext@@UAAXPAUwavehdr_tag@@@Z 100057a0 f   wavedev2_common_topaz_v1:strmctxt.obj
 0001:000047e0       ?DoCallbackStreamOpened@StreamContext@@UAAXXZ 100057e0 f   wavedev2_common_topaz_v1:strmctxt.obj
 0001:00004820       ?DoCallbackStreamClosed@StreamContext@@UAAXXZ 10005820 f   wavedev2_common_topaz_v1:strmctxt.obj
 0001:0000485c       ?GetGain@StreamContext@@QAAKXZ 1000585c f   wavedev2_common_topaz_v1:strmctxt.obj
 0001:00004864       ?SetGain@StreamContext@@QAAKK@Z 10005864 f   wavedev2_common_topaz_v1:strmctxt.obj
 0001:0000488c       ?SetSecondaryGainClass@StreamContext@@QAAKK@Z 1000588c f   wavedev2_common_topaz_v1:strmctxt.obj
 0001:000048c8       ?IsExclusive@StreamContext@@UAAHXZ 100058c8 f   wavedev2_common_topaz_v1:strmctxt.obj
 0001:000048d0       ?Open@StreamContext@@UAAKPAVDeviceContext@@PAUwaveopendesc_tag@@K@Z 100058d0 f   wavedev2_common_topaz_v1:strmctxt.obj
 0001:00004a38       ?AddRef@StreamContext@@QAAJXZ 10005a38 f   wavedev2_common_topaz_v1:strmctxt.obj
 0001:00004a4c       ?Release@StreamContext@@QAAJXZ 10005a4c f   wavedev2_common_topaz_v1:strmctxt.obj
 0001:00004a98       ?QueueBuffer@StreamContext@@UAAKPAUwavehdr_tag@@@Z 10005a98 f   wavedev2_common_topaz_v1:strmctxt.obj
 0001:00004b48       ?GetNextBuffer@StreamContext@@QAAPAEXZ 10005b48 f   wavedev2_common_topaz_v1:strmctxt.obj
 0001:00004c24       ?BreakLoop@StreamContext@@QAAKXZ 10005c24 f   wavedev2_common_topaz_v1:strmctxt.obj
 0001:00004cb4       ?MapGain@StreamContext@@QAAKKK@Z 10005cb4 f   wavedev2_common_topaz_v1:strmctxt.obj
 0001:00004d7c       ?GetPos@StreamContext@@UAAKPAUmmtime_tag@@@Z 10005d7c f   wavedev2_common_topaz_v1:strmctxt.obj
 0001:00004e60       ?Open@WaveStreamContext@@UAAKPAVDeviceContext@@PAUwaveopendesc_tag@@K@Z 10005e60 f   wavedev2_common_topaz_v1:strmctxt.obj
 0001:00004f94       ?GetRate@WaveStreamContext@@QAAKPAK@Z 10005f94 f   wavedev2_common_topaz_v1:strmctxt.obj
 0001:00004fa4       ?Run@StreamContext@@UAAKXZ 10005fa4 f   wavedev2_common_topaz_v1:strmctxt.obj
 0001:00004fdc       ?Stop@StreamContext@@UAAKXZ 10005fdc f   wavedev2_common_topaz_v1:strmctxt.obj
 0001:00004fec       ?Reset@StreamContext@@UAAKXZ 10005fec f   wavedev2_common_topaz_v1:strmctxt.obj
 0001:00005088       ?ForceSpeaker@StreamContext@@QAAKH@Z 10006088 f   wavedev2_common_topaz_v1:strmctxt.obj
 0001:000050c8       ?SetRate@WaveStreamContext@@UAAKK@Z 100060c8 f   wavedev2_common_topaz_v1:strmctxt.obj
 0001:00005130       ?Render@WaveStreamContext@@UAAPAEPAE00PAUTRANSFER_STATUS@@@Z 10006130 f   wavedev2_common_topaz_v1:strmctxt.obj
 0001:00005224       ?ClearBuffer@StreamContext@@SAXPAE0@Z 10006224 f   wavedev2_common_topaz_v1:strmctxt.obj
 0001:0000523c       ?GetProperty@StreamContext@@QAAKPAUtag_WAVEPROPINFO@@@Z 1000623c f   wavedev2_common_topaz_v1:strmctxt.obj
 0001:00005250       ?SetProperty@StreamContext@@QAAKPAUtag_WAVEPROPINFO@@@Z 10006250 f   wavedev2_common_topaz_v1:strmctxt.obj
 0001:00005264       ??_GStreamContext@@UAAPAXI@Z 10006264 f i wavedev2_common_topaz_v1:strmctxt.obj
 0001:00005264       ??_EStreamContext@@UAAPAXI@Z 10006264 f i wavedev2_common_topaz_v1:strmctxt.obj
 0001:0000528c       ?GainChange@StreamContext@@UAAXXZ 1000628c f   wavedev2_common_topaz_v1:strmctxt.obj
 0001:000052c8       ?Close@StreamContext@@UAAKXZ 100062c8 f   wavedev2_common_topaz_v1:strmctxt.obj
 0001:00005328       ?LookupMxLine@@YAPBUtagMXLINEDESC@@G@Z 10006328 f   wavedev2_common_topaz_v1:mixerdrv.obj
 0001:00005374       ?SetControlID@MixerControl@@UAAXK@Z 10006374 f i wavedev2_common_topaz_v1:mixerdrv.obj
 0001:0000537c       ?CopyMixerControl@MixerControl@@UAAXPAUtMIXERCONTROL@@@Z 1000637c f i wavedev2_common_topaz_v1:mixerdrv.obj
 0001:000053f4       ?GetControlDetails@MixerControl@@UAAKPAUtMIXERCONTROLDETAILS@@K@Z 100063f4 f i wavedev2_common_topaz_v1:mixerdrv.obj
 0001:000053fc       ?SetControlDetails@MixerControl@@UAAKPAUtMIXERCONTROLDETAILS@@K@Z 100063fc f i wavedev2_common_topaz_v1:mixerdrv.obj
 0001:00005404       ??_GMixerControl@@UAAPAXI@Z 10006404 f i wavedev2_common_topaz_v1:mixerdrv.obj
 0001:00005404       ??_EMixerControl@@UAAPAXI@Z 10006404 f i wavedev2_common_topaz_v1:mixerdrv.obj
 0001:0000542c       ?CopyMixerControl@MixerControlVolume@@UAAXPAUtMIXERCONTROL@@@Z 1000642c f i wavedev2_common_topaz_v1:mixerdrv.obj
 0001:0000549c       ?GetControlType@MixerControlVolume@@UAAKXZ 1000649c f i wavedev2_common_topaz_v1:mixerdrv.obj
 0001:000054a8       ?GetControlDetails@MixerControlVolume@@UAAKPAUtMIXERCONTROLDETAILS@@K@Z 100064a8 f i wavedev2_common_topaz_v1:mixerdrv.obj
 0001:000055a0       ?SetControlDetails@MixerControlVolume@@UAAKPAUtMIXERCONTROLDETAILS@@K@Z 100065a0 f i wavedev2_common_topaz_v1:mixerdrv.obj
 0001:00005698       ?CopyMixerControl@MixerControlVolumeMaster@@UAAXPAUtMIXERCONTROL@@@Z 10006698 f i wavedev2_common_topaz_v1:mixerdrv.obj
 0001:000056c8       ?GetLineID@MixerControlVolumeMaster@@UAAGXZ 100066c8 f i wavedev2_common_topaz_v1:mixerdrv.obj
 0001:000056d4       ?SetGain@MixerControlVolumeMaster@@UAAXK@Z 100066d4 f i wavedev2_common_topaz_v1:mixerdrv.obj
 0001:000056f0       ?GetGain@MixerControlVolumeMaster@@UAAKXZ 100066f0 f i wavedev2_common_topaz_v1:mixerdrv.obj
 0001:0000570c       ?CopyMixerControl@MixerControlVolumeMic@@UAAXPAUtMIXERCONTROL@@@Z 1000670c f i wavedev2_common_topaz_v1:mixerdrv.obj
 0001:0000573c       ?GetLineID@MixerControlVolumeMic@@UAAGXZ 1000673c f i wavedev2_common_topaz_v1:mixerdrv.obj
 0001:00005748       ?SetGain@MixerControlVolumeMic@@UAAXK@Z 10006748 f i wavedev2_common_topaz_v1:mixerdrv.obj
 0001:00005764       ?GetGain@MixerControlVolumeMic@@UAAKXZ 10006764 f i wavedev2_common_topaz_v1:mixerdrv.obj
 0001:00005780       ?CopyMixerControl@MixerControlBoolean@@UAAXPAUtMIXERCONTROL@@@Z 10006780 f i wavedev2_common_topaz_v1:mixerdrv.obj
 0001:000057ec       ?GetControlType@MixerControlBoolean@@UAAKXZ 100067ec f i wavedev2_common_topaz_v1:mixerdrv.obj
 0001:000057f8       ?GetControlDetails@MixerControlBoolean@@UAAKPAUtMIXERCONTROLDETAILS@@K@Z 100067f8 f i wavedev2_common_topaz_v1:mixerdrv.obj
 0001:00005854       ?SetControlDetails@MixerControlBoolean@@UAAKPAUtMIXERCONTROLDETAILS@@K@Z 10006854 f i wavedev2_common_topaz_v1:mixerdrv.obj
 0001:000058ac       ?CopyMixerControl@MixerControlMuteMaster@@UAAXPAUtMIXERCONTROL@@@Z 100068ac f i wavedev2_common_topaz_v1:mixerdrv.obj
 0001:000058dc       ?GetControlType@MixerControlMuteMaster@@UAAKXZ 100068dc f i wavedev2_common_topaz_v1:mixerdrv.obj
 0001:000058e8       ?GetLineID@MixerControlMuteMaster@@UAAGXZ 100068e8 f i wavedev2_common_topaz_v1:mixerdrv.obj
 0001:000058f4       ?GetValue@MixerControlMuteMaster@@UAAHXZ 100068f4 f i wavedev2_common_topaz_v1:mixerdrv.obj
 0001:00005910       ?SetValue@MixerControlMuteMaster@@UAAXH@Z 10006910 f i wavedev2_common_topaz_v1:mixerdrv.obj
 0001:0000592c       ?CopyMixerControl@MixerControlMuteMic@@UAAXPAUtMIXERCONTROL@@@Z 1000692c f i wavedev2_common_topaz_v1:mixerdrv.obj
 0001:0000595c       ?GetLineID@MixerControlMuteMic@@UAAGXZ 1000695c f i wavedev2_common_topaz_v1:mixerdrv.obj
 0001:00005968       ?GetValue@MixerControlMuteMic@@UAAHXZ 10006968 f i wavedev2_common_topaz_v1:mixerdrv.obj
 0001:00005984       ?SetValue@MixerControlMuteMic@@UAAXH@Z 10006984 f i wavedev2_common_topaz_v1:mixerdrv.obj
 0001:000059a0       ?CopyMixerControl@MixerControlLoopback@@UAAXPAUtMIXERCONTROL@@@Z 100069a0 f i wavedev2_common_topaz_v1:mixerdrv.obj
 0001:000059d4       ?GetControlType@MixerControlLoopback@@UAAKXZ 100069d4 f i wavedev2_common_topaz_v1:mixerdrv.obj
 0001:000059e0       ?GetLineID@MixerControlLoopback@@UAAGXZ 100069e0 f i wavedev2_common_topaz_v1:mixerdrv.obj
 0001:000059ec       ?GetValue@MixerControlLoopback@@UAAHXZ 100069ec f i wavedev2_common_topaz_v1:mixerdrv.obj
 0001:000059f4       ?SetValue@MixerControlLoopback@@UAAXH@Z 100069f4 f i wavedev2_common_topaz_v1:mixerdrv.obj
 0001:00005a2c       ?GetLineID@MixerControlInputMux@@UAAGXZ 10006a2c f i wavedev2_common_topaz_v1:mixerdrv.obj
 0001:00005a38       ?GetControlType@MixerControlInputMux@@UAAKXZ 10006a38 f i wavedev2_common_topaz_v1:mixerdrv.obj
 0001:00005a44       ?GetListText@MixerControlInputMux@@QAAXPAUtMIXERCONTROLDETAILS_LISTTEXT@@K@Z 10006a44 f i wavedev2_common_topaz_v1:mixerdrv.obj
 0001:00005ae8       ?GetControlDetails@MixerControlInputMux@@UAAKPAUtMIXERCONTROLDETAILS@@K@Z 10006ae8 f i wavedev2_common_topaz_v1:mixerdrv.obj
 0001:00005c20       ?SetControlDetails@MixerControlInputMux@@UAAKPAUtMIXERCONTROLDETAILS@@K@Z 10006c20 f i wavedev2_common_topaz_v1:mixerdrv.obj
 0001:00005d0c       ??0MixerControlList@@QAA@XZ 10006d0c f i wavedev2_common_topaz_v1:mixerdrv.obj
 0001:00005de4       ??_EMixerControlList@@UAAPAXI@Z 10006de4 f i wavedev2_common_topaz_v1:mixerdrv.obj
 0001:00005de4       ??_GMixerControlList@@UAAPAXI@Z 10006de4 f i wavedev2_common_topaz_v1:mixerdrv.obj
 0001:00005e2c       ?PerformMixerCallbacks@@YAXKK@Z 10006e2c f   wavedev2_common_topaz_v1:mixerdrv.obj
 0001:00005e90       ?wdev_MXDM_GETDEVCAPS@@YAKPAUtagMIXERCAPS@@K@Z 10006e90 f   wavedev2_common_topaz_v1:mixerdrv.obj
 0001:00005f04       ?wdev_MXDM_OPEN@@YAKPAKPAUtMIXEROPENDESC@@K@Z 10006f04 f   wavedev2_common_topaz_v1:mixerdrv.obj
 0001:00005f9c       ?wdev_MXDM_CLOSE@@YAKK@Z   10006f9c f   wavedev2_common_topaz_v1:mixerdrv.obj
 0001:00005ff4       ?wdev_MXDM_GETLINEINFO@@YAKPAUtMIXERLINE@@K@Z 10006ff4 f   wavedev2_common_topaz_v1:mixerdrv.obj
 0001:00006368       ?wdev_MXDM_GETLINECONTROLS@@YAKPAUtMIXERLINECONTROLS@@K@Z 10007368 f   wavedev2_common_topaz_v1:mixerdrv.obj
 0001:000065f8       ?wdev_MXDM_GETCONTROLDETAILS@@YAKPAUtMIXERCONTROLDETAILS@@K@Z 100075f8 f   wavedev2_common_topaz_v1:mixerdrv.obj
 0001:00006670       ?wdev_MXDM_SETCONTROLDETAILS@@YAKPAUtMIXERCONTROLDETAILS@@K@Z 10007670 f   wavedev2_common_topaz_v1:mixerdrv.obj
 0001:00006714       ?InitMixerControls@@YAHXZ  10007714 f   wavedev2_common_topaz_v1:mixerdrv.obj
 0001:0000675c       ?HandleMixerMessage@@YAHPAUMMDRV_MESSAGE_PARAMS@@PAK@Z 1000775c f   wavedev2_common_topaz_v1:mixerdrv.obj
 0001:00006854       ?SetMasterVolume@@YAIK@Z   10007854 f   wavedev2_common_topaz_v1:mixerdrv.obj
 0001:0000689c       ?GetMasterVolume@@YAKXZ    1000789c f   wavedev2_common_topaz_v1:mixerdrv.obj
 0001:000068c8       ??_GMixerControlVolumeMaster@@UAAPAXI@Z 100078c8 f i wavedev2_common_topaz_v1:mixerdrv.obj
 0001:000068c8       ??_EMixerControlVolumeMaster@@UAAPAXI@Z 100078c8 f i wavedev2_common_topaz_v1:mixerdrv.obj
 0001:000068f0       ??_EMixerControlVolumeMic@@UAAPAXI@Z 100078f0 f i wavedev2_common_topaz_v1:mixerdrv.obj
 0001:000068f0       ??_GMixerControlVolumeMic@@UAAPAXI@Z 100078f0 f i wavedev2_common_topaz_v1:mixerdrv.obj
 0001:00006918       ??_GMixerControlMuteMaster@@UAAPAXI@Z 10007918 f i wavedev2_common_topaz_v1:mixerdrv.obj
 0001:00006918       ??_EMixerControlMuteMaster@@UAAPAXI@Z 10007918 f i wavedev2_common_topaz_v1:mixerdrv.obj
 0001:00006940       ??_GMixerControlMuteMic@@UAAPAXI@Z 10007940 f i wavedev2_common_topaz_v1:mixerdrv.obj
 0001:00006940       ??_EMixerControlMuteMic@@UAAPAXI@Z 10007940 f i wavedev2_common_topaz_v1:mixerdrv.obj
 0001:00006968       ??_GMixerControlLoopback@@UAAPAXI@Z 10007968 f i wavedev2_common_topaz_v1:mixerdrv.obj
 0001:00006968       ??_EMixerControlLoopback@@UAAPAXI@Z 10007968 f i wavedev2_common_topaz_v1:mixerdrv.obj
 0001:00006990       ?CopyMixerControl@MixerControlInputMux@@UAAXPAUtMIXERCONTROL@@@Z 10007990 f i wavedev2_common_topaz_v1:mixerdrv.obj
 0001:00006a20       ??_GMixerControlInputMux@@UAAPAXI@Z 10007a20 f i wavedev2_common_topaz_v1:mixerdrv.obj
 0001:00006a20       ??_EMixerControlInputMux@@UAAPAXI@Z 10007a20 f i wavedev2_common_topaz_v1:mixerdrv.obj
 0001:00006a48       ?GainChange@CMidiStream@@UAAXXZ 10007a48 f   wavedev2_common_topaz_v1:midistrm.obj
 0001:00006a78       ?MapNoteGain@CMidiStream@@QAAKKK@Z 10007a78 f   wavedev2_common_topaz_v1:midistrm.obj
 0001:00006abc       ?Open@CMidiStream@@UAAKPAVDeviceContext@@PAUwaveopendesc_tag@@K@Z 10007abc f   wavedev2_common_topaz_v1:midistrm.obj
 0001:00006ba8       ?UpdateTempo@CMidiStream@@QAAJXZ 10007ba8 f   wavedev2_common_topaz_v1:midistrm.obj
 0001:00006c08       ?FindNote@CMidiStream@@QAAPAVCMidiNote@@II@Z 10007c08 f   wavedev2_common_topaz_v1:midistrm.obj
 0001:00006c60       ?AllNotesOff@CMidiStream@@QAAJI@Z 10007c60 f   wavedev2_common_topaz_v1:midistrm.obj
 0001:00006c9c       ?ResetBaseInfo@CMidiStream@@UAAXXZ 10007c9c f   wavedev2_common_topaz_v1:midistrm.obj
 0001:00006d24       ?GetDeltaFromNote@CMidiStream@@QAAKK@Z 10007d24 f   wavedev2_common_topaz_v1:midistrm.obj
 0001:00006d70       ?GetDeltaFromFreq@CMidiStream@@QAAKK@Z 10007d70 f   wavedev2_common_topaz_v1:midistrm.obj
 0001:00006d90       ?NoteDone@CMidiStream@@QAAXPAVCMidiNote@@@Z 10007d90 f   wavedev2_common_topaz_v1:midistrm.obj
 0001:00006dd4       ?Reset@CMidiStream@@UAAKXZ 10007dd4 f   wavedev2_common_topaz_v1:midistrm.obj
 0001:00006e14       ?Close@CMidiStream@@UAAKXZ 10007e14 f   wavedev2_common_topaz_v1:midistrm.obj
 0001:00006e3c       ?NoteOn@CMidiStream@@QAAJIII@Z 10007e3c f   wavedev2_common_topaz_v1:midistrm.obj
 0001:00006ef4       ?MidiData@CMidiStream@@QAAJI@Z 10007ef4 f   wavedev2_common_topaz_v1:midistrm.obj
 0001:00006fa8       ?InternalMidiMessage@CMidiStream@@QAAJI@Z 10007fa8 f   wavedev2_common_topaz_v1:midistrm.obj
 0001:00007058       ?ProcessMidiStream@CMidiStream@@QAAIXZ 10008058 f   wavedev2_common_topaz_v1:midistrm.obj
 0001:00007128       ?Render@CMidiStream@@UAAPAEPAE00PAUTRANSFER_STATUS@@@Z 10008128 f   wavedev2_common_topaz_v1:midistrm.obj
 0001:00007254       ?Open@OutputStreamContext@@UAAKPAVDeviceContext@@PAUwaveopendesc_tag@@K@Z 10008254 f   wavedev2_common_topaz_v1:output.obj
 0001:00007298       ?Reset@OutputStreamContext@@UAAKXZ 10008298 f   wavedev2_common_topaz_v1:output.obj
 0001:000072c8       ?ResetBaseInfo@OutputStreamContext@@UAAXXZ 100082c8 f   wavedev2_common_topaz_v1:output.obj
 0001:000072cc       ?Render2@OutputStreamContext16bitM8@@UAAPAEPAE00PAUTRANSFER_STATUS@@@Z 100082cc f   wavedev2_common_topaz_v1:output.obj
 0001:00007458       ?Render2@OutputStreamContext16bitM16@@UAAPAEPAE00PAUTRANSFER_STATUS@@@Z 10008458 f   wavedev2_common_topaz_v1:output.obj
 0001:000075e0       ?Render2@OutputStreamContext16bitS8@@UAAPAEPAE00PAUTRANSFER_STATUS@@@Z 100085e0 f   wavedev2_common_topaz_v1:output.obj
 0001:000077c4       ?Render2@OutputStreamContext16bitS16@@UAAPAEPAE00PAUTRANSFER_STATUS@@@Z 100087c4 f   wavedev2_common_topaz_v1:output.obj
 0001:00007a48       ?Render2@OutputStreamContext24bitM8@@UAAPAEPAE00PAUTRANSFER_STATUS@@@Z 10008a48 f   wavedev2_common_topaz_v1:output.obj
 0001:00007c38       ?Render2@OutputStreamContext24bitM16@@UAAPAEPAE00PAUTRANSFER_STATUS@@@Z 10008c38 f   wavedev2_common_topaz_v1:output.obj
 0001:00007e10       ?Render2@OutputStreamContext24bitS8@@UAAPAEPAE00PAUTRANSFER_STATUS@@@Z 10008e10 f   wavedev2_common_topaz_v1:output.obj
 0001:00008040       ?Render2@OutputStreamContext24bitS16@@UAAPAEPAE00PAUTRANSFER_STATUS@@@Z 10009040 f   wavedev2_common_topaz_v1:output.obj
 0001:00008370       ?Render2@OutputStreamContext24bitS24@@UAAPAEPAE00PAUTRANSFER_STATUS@@@Z 10009370 f   wavedev2_common_topaz_v1:output.obj
 0001:000085cc       ?Open@InputStreamContext@@UAAKPAVDeviceContext@@PAUwaveopendesc_tag@@K@Z 100095cc f   wavedev2_common_topaz_v1:input.obj
 0001:000085ec       ?DoCallbackReturnBuffer@InputStreamContext@@UAAXPAUwavehdr_tag@@@Z 100095ec f   wavedev2_common_topaz_v1:input.obj
 0001:00008608       ?DoCallbackStreamOpened@InputStreamContext@@UAAXXZ 10009608 f   wavedev2_common_topaz_v1:input.obj
 0001:00008628       ?DoCallbackStreamClosed@InputStreamContext@@UAAXXZ 10009628 f   wavedev2_common_topaz_v1:input.obj
 0001:00008648       ?Stop@InputStreamContext@@UAAKXZ 10009648 f   wavedev2_common_topaz_v1:input.obj
 0001:0000867c       ?Render2@InputStreamContext@@UAAPAEPAE00PAUTRANSFER_STATUS@@@Z 1000967c f   wavedev2_common_topaz_v1:input.obj
 0001:00008904       ?ResetBaseInfo@InputStreamContext@@UAAXXZ 10009904 f   wavedev2_common_topaz_v1:input.obj
 0001:00008908       ?GainChange@CMidiNote@@QAAXXZ 10009908 f   wavedev2_common_topaz_v1:midinote.obj
 0001:00008944       ?ResetBaseInfo@CMidiNote@@QAAXXZ 10009944 f   wavedev2_common_topaz_v1:midinote.obj
 0001:00008978       ?NoteOff@CMidiNote@@QAAJI@Z 10009978 f   wavedev2_common_topaz_v1:midinote.obj
 0001:000089d4       ?Render2@CMidiNote@@QAAPAEPAE00PAUTRANSFER_STATUS@@@Z 100099d4 f   wavedev2_common_topaz_v1:midinote.obj
 0001:00008bb8       ?NoteVal@CMidiNote@@QAAIXZ 10009bb8 f   wavedev2_common_topaz_v1:midinote.obj
 0001:00008bc0       ?NoteChannel@CMidiNote@@QAAIXZ 10009bc0 f   wavedev2_common_topaz_v1:midinote.obj
 0001:00008bc8       ?SetVelocity@CMidiNote@@QAAXI@Z 10009bc8 f   wavedev2_common_topaz_v1:midinote.obj
 0001:00008bf4       ?NoteOn@CMidiNote@@QAAJPAVCMidiStream@@III@Z 10009bf4 f   wavedev2_common_topaz_v1:midinote.obj
 0001:00008c44       ?Render@CMidiNote@@QAAPAEPAE00PAUTRANSFER_STATUS@@@Z 10009c44 f   wavedev2_common_topaz_v1:midinote.obj
 0001:00008cd0       ?GetSsiBaseRegAddr@@YAII@Z 10009cd0 f   wavedev2_mx25_topaz_v1:csphwctxt.obj
 0001:00008cf8       ?GetAudmuxBaseRegAddr@@YAIXZ 10009cf8 f   wavedev2_mx25_topaz_v1:csphwctxt.obj
 0001:00008d04       ?GetSdmaChannelIRQ@@YAKI@Z 10009d04 f   wavedev2_mx25_topaz_v1:csphwctxt.obj
 0001:00008d0c       DeleteCriticalSection      10009d0c f   coredll:COREDLL.dll
 0001:00008d1c       LeaveCriticalSection       10009d1c f   coredll:COREDLL.dll
 0001:00008d2c       EnterCriticalSection       10009d2c f   coredll:COREDLL.dll
 0001:00008d3c       InitializeCriticalSection  10009d3c f   coredll:COREDLL.dll
 0001:00008d4c       Sleep                      10009d4c f   coredll:COREDLL.dll
 0001:00008d5c       DisableThreadLibraryCalls  10009d5c f   coredll:COREDLL.dll
 0001:00008d6c       SetLastError               10009d6c f   coredll:COREDLL.dll
 0001:00008d7c       CeGetCallerTrust           10009d7c f   coredll:COREDLL.dll
 0001:00008d8c       EventModify                10009d8c f   coredll:COREDLL.dll
 0001:00008d9c       CloseHandle                10009d9c f   coredll:COREDLL.dll
 0001:00008dac       KernelIoControl            10009dac f   coredll:COREDLL.dll
 0001:00008dbc       InterruptDone              10009dbc f   coredll:COREDLL.dll
 0001:00008dcc       WaitForSingleObject        10009dcc f   coredll:COREDLL.dll
 0001:00008ddc       WaitForMultipleObjects     10009ddc f   coredll:COREDLL.dll
 0001:00008dec       RegCloseKey                10009dec f   coredll:COREDLL.dll
 0001:00008dfc       RegQueryValueExW           10009dfc f   coredll:COREDLL.dll
 0001:00008e0c       OpenDeviceKey              10009e0c f   coredll:COREDLL.dll
 0001:00008e1c       CreateThread               10009e1c f   coredll:COREDLL.dll
 0001:00008e2c       InterruptInitialize        10009e2c f   coredll:COREDLL.dll
 0001:00008e3c       CreateEventW               10009e3c f   coredll:COREDLL.dll
 0001:00008e4c       CeSetThreadPriority        10009e4c f   coredll:COREDLL.dll
 0001:00008e5c       CeSafeCopyMemory           10009e5c f   coredll:COREDLL.dll
 0001:00008e6c       LocalAlloc                 10009e6c f   coredll:COREDLL.dll
 0001:00008e7c       LocalFree                  10009e7c f   coredll:COREDLL.dll
 0001:00008e8c       MmMapIoSpace               10009e8c f   ceddk:CEDDK.dll
 0001:00008e9c       HalAllocateCommonBuffer    10009e9c f   ceddk:CEDDK.dll
 0001:00008eac       HalFreeCommonBuffer        10009eac f   ceddk:CEDDK.dll
 0001:00008ebc       MmUnmapIoSpace             10009ebc f   ceddk:CEDDK.dll
 0001:00008ecc       timeSetEvent               10009ecc f   mmtimer:MMTimer.dll
 0001:00008edc       timeKillEvent              10009edc f   mmtimer:MMTimer.dll
 0001:00008eec       DDKIomuxSetPinMux          10009eec f   cspddk:CSPDDK.dll
 0001:00008efc       DDKClockSetGatingMode      10009efc f   cspddk:CSPDDK.dll
 0001:00008f0c       DDKClockSetCKO             10009f0c f   cspddk:CSPDDK.dll
 0001:00008f1c       DDKSdmaSetBufDesc          10009f1c f   cspddk:CSPDDK.dll
 0001:00008f2c       DDKSdmaAllocChain          10009f2c f   cspddk:CSPDDK.dll
 0001:00008f3c       DDKSdmaOpenChan            10009f3c f   cspddk:CSPDDK.dll
 0001:00008f4c       DDKSdmaStopChan            10009f4c f   cspddk:CSPDDK.dll
 0001:00008f5c       DDKSdmaStartChan           10009f5c f   cspddk:CSPDDK.dll
 0001:00008f6c       DDKSdmaInitChain           10009f6c f   cspddk:CSPDDK.dll
 0001:00008f7c       DDKSdmaClearBufDescStatus  10009f7c f   cspddk:CSPDDK.dll
 0001:00008f8c       DDKSdmaGetChainStatus      10009f8c f   cspddk:CSPDDK.dll
 0001:00008f9c       I2CCloseHandle             10009f9c f   i2csdk:I2CSDK.dll
 0001:00008fac       I2CTransfer                10009fac f   i2csdk:I2CSDK.dll
 0001:00008fbc       I2CSetFrequency            10009fbc f   i2csdk:I2CSDK.dll
 0001:00008fcc       I2CSetMasterMode           10009fcc f   i2csdk:I2CSDK.dll
 0001:00008fdc       I2COpenHandle              10009fdc f   i2csdk:I2CSDK.dll
 0001:000090f0       _DllMainCRTStartup         1000a0f0 f   corelib0:pegdmain.obj
 0001:0000921c       _cexit                     1000a21c f   corelib0:cexit.obj
 0001:00009238       _initterm                  1000a238 f   corelib0:crt0dat.obj
 0001:0000926c       _cinit                     1000a26c f   corelib0:crt0dat.obj
 0001:000092a0       __security_init_cookie     1000a2a0 f   corelib0:seccinit.obj
 0001:000092fc       __utod                     1000a2fc f   corelib1:COREDLL.dll
 0001:0000930c       log                        1000a30c f   corelib1:COREDLL.dll
 0001:0000931c       __subd                     1000a31c f   corelib1:COREDLL.dll
 0001:0000932c       __muld                     1000a32c f   corelib1:COREDLL.dll
 0001:0000933c       __divd                     1000a33c f   corelib1:COREDLL.dll
 0001:0000934c       __addd                     1000a34c f   corelib1:COREDLL.dll
 0001:0000935c       __dtou                     1000a35c f   corelib1:COREDLL.dll
 0001:0000936c       ??3@YAXPAX@Z               1000a36c f   corelib1:COREDLL.dll
 0001:0000937c       ??2@YAPAXI@Z               1000a37c f   corelib1:COREDLL.dll
 0001:0000938c       __C_specific_handler       1000a38c f   corelib1:COREDLL.dll
 0001:0000939c       memset                     1000a39c f   corelib1:COREDLL.dll
 0001:000093ac       memcmp                     1000a3ac f   corelib1:COREDLL.dll
 0001:000093bc       _purecall                  1000a3bc f   corelib1:COREDLL.dll
 0001:000093cc       memcpy                     1000a3cc f   corelib1:COREDLL.dll
 0001:000093dc       __rt_sdiv64by64            1000a3dc f   corelib1:COREDLL.dll
 0001:000093ec       __rt_udiv                  1000a3ec f   corelib1:COREDLL.dll
 0001:000093fc       wcscpy                     1000a3fc f   corelib1:COREDLL.dll
 0001:0000940c       __rt_udiv64by64            1000a40c f   corelib1:COREDLL.dll
 0001:0000941c       _XcptFilter                1000a41c f   corelib1:COREDLL.dll
 0001:0000942c       free                       1000a42c f   corelib1:COREDLL.dll
 0001:0000943c       __security_gen_cookie2     1000a43c f   corelib1:COREDLL.dll
 0001:0000944c       InterlockedExchange        1000a44c f   coredll:COREDLL.dll
 0001:0000945c       TerminateProcess           1000a45c f   coredll:COREDLL.dll
 0001:000094d0       __IMPORT_DESCRIPTOR_COREDLL 1000a4d0     coredll:COREDLL.dll
 0001:000094e4       __IMPORT_DESCRIPTOR_CEDDK  1000a4e4     ceddk:CEDDK.dll
 0001:000094f8       __IMPORT_DESCRIPTOR_MMTimer 1000a4f8     mmtimer:MMTimer.dll
 0001:0000950c       __IMPORT_DESCRIPTOR_CSPDDK 1000a50c     cspddk:CSPDDK.dll
 0001:00009520       __IMPORT_DESCRIPTOR_I2CSDK 1000a520     i2csdk:I2CSDK.dll
 0001:00009534       __NULL_IMPORT_DESCRIPTOR   1000a534     coredll:COREDLL.dll
 0002:00000000       __imp_HalFreeCommonBuffer  1000b000     ceddk:CEDDK.dll
 0002:00000004       __imp_HalAllocateCommonBuffer 1000b004     ceddk:CEDDK.dll
 0002:00000008       __imp_MmMapIoSpace         1000b008     ceddk:CEDDK.dll
 0002:0000000c       __imp_MmUnmapIoSpace       1000b00c     ceddk:CEDDK.dll
 0002:00000010       \177CEDDK_NULL_THUNK_DATA  1000b010     ceddk:CEDDK.dll
 0002:00000014       __imp_DisableThreadLibraryCalls 1000b014     coredll:COREDLL.dll
 0002:00000018       __imp_SetLastError         1000b018     coredll:COREDLL.dll
 0002:0000001c       __imp_CeGetCallerTrust     1000b01c     coredll:COREDLL.dll
 0002:00000020       __imp_EventModify          1000b020     coredll:COREDLL.dll
 0002:00000024       __imp_CloseHandle          1000b024     coredll:COREDLL.dll
 0002:00000028       __imp_KernelIoControl      1000b028     coredll:COREDLL.dll
 0002:0000002c       __imp_InterruptDone        1000b02c     coredll:COREDLL.dll
 0002:00000030       __imp_WaitForSingleObject  1000b030     coredll:COREDLL.dll
 0002:00000034       __imp_WaitForMultipleObjects 1000b034     coredll:COREDLL.dll
 0002:00000038       __imp_RegCloseKey          1000b038     coredll:COREDLL.dll
 0002:0000003c       __imp_Sleep                1000b03c     coredll:COREDLL.dll
 0002:00000040       __imp_OpenDeviceKey        1000b040     coredll:COREDLL.dll
 0002:00000044       __imp_CreateThread         1000b044     coredll:COREDLL.dll
 0002:00000048       __imp_InterruptInitialize  1000b048     coredll:COREDLL.dll
 0002:0000004c       __imp_CreateEventW         1000b04c     coredll:COREDLL.dll
 0002:00000050       __imp_CeSetThreadPriority  1000b050     coredll:COREDLL.dll
 0002:00000054       __imp_CeSafeCopyMemory     1000b054     coredll:COREDLL.dll
 0002:00000058       __imp_LocalAlloc           1000b058     coredll:COREDLL.dll
 0002:0000005c       __imp_LocalFree            1000b05c     coredll:COREDLL.dll
 0002:00000060       __imp_InitializeCriticalSection 1000b060     coredll:COREDLL.dll
 0002:00000064       __imp_EnterCriticalSection 1000b064     coredll:COREDLL.dll
 0002:00000068       __imp_LeaveCriticalSection 1000b068     coredll:COREDLL.dll
 0002:0000006c       __imp_RegQueryValueExW     1000b06c     coredll:COREDLL.dll
 0002:00000070       __imp_DeleteCriticalSection 1000b070     coredll:COREDLL.dll
 0002:00000074       __imp_TerminateProcess     1000b074     coredll:COREDLL.dll
 0002:00000078       __imp_InterlockedExchange  1000b078     coredll:COREDLL.dll
 0002:0000007c       __imp___security_gen_cookie2 1000b07c     corelib1:COREDLL.dll
 0002:00000080       __imp_free                 1000b080     corelib1:COREDLL.dll
 0002:00000084       __imp__XcptFilter          1000b084     corelib1:COREDLL.dll
 0002:00000088       __imp___rt_udiv64by64      1000b088     corelib1:COREDLL.dll
 0002:0000008c       __imp_wcscpy               1000b08c     corelib1:COREDLL.dll
 0002:00000090       __imp___rt_udiv            1000b090     corelib1:COREDLL.dll
 0002:00000094       __imp___rt_sdiv64by64      1000b094     corelib1:COREDLL.dll
 0002:00000098       __imp_memcpy               1000b098     corelib1:COREDLL.dll
 0002:0000009c       __imp__purecall            1000b09c     corelib1:COREDLL.dll
 0002:000000a0       __imp_memcmp               1000b0a0     corelib1:COREDLL.dll
 0002:000000a4       __imp_memset               1000b0a4     corelib1:COREDLL.dll
 0002:000000a8       __imp___C_specific_handler 1000b0a8     corelib1:COREDLL.dll
 0002:000000ac       __imp_??2@YAPAXI@Z         1000b0ac     corelib1:COREDLL.dll
 0002:000000b0       __imp_??3@YAXPAX@Z         1000b0b0     corelib1:COREDLL.dll
 0002:000000b4       __imp___dtou               1000b0b4     corelib1:COREDLL.dll
 0002:000000b8       __imp___utod               1000b0b8     corelib1:COREDLL.dll
 0002:000000bc       __imp_log                  1000b0bc     corelib1:COREDLL.dll
 0002:000000c0       __imp___subd               1000b0c0     corelib1:COREDLL.dll
 0002:000000c4       __imp___muld               1000b0c4     corelib1:COREDLL.dll
 0002:000000c8       __imp___divd               1000b0c8     corelib1:COREDLL.dll
 0002:000000cc       __imp___addd               1000b0cc     corelib1:COREDLL.dll
 0002:000000d0       \177COREDLL_NULL_THUNK_DATA 1000b0d0     coredll:COREDLL.dll
 0002:000000d4       __imp_DDKSdmaStartChan     1000b0d4     cspddk:CSPDDK.dll
 0002:000000d8       __imp_DDKIomuxSetPinMux    1000b0d8     cspddk:CSPDDK.dll
 0002:000000dc       __imp_DDKClockSetGatingMode 1000b0dc     cspddk:CSPDDK.dll
 0002:000000e0       __imp_DDKClockSetCKO       1000b0e0     cspddk:CSPDDK.dll
 0002:000000e4       __imp_DDKSdmaSetBufDesc    1000b0e4     cspddk:CSPDDK.dll
 0002:000000e8       __imp_DDKSdmaAllocChain    1000b0e8     cspddk:CSPDDK.dll
 0002:000000ec       __imp_DDKSdmaGetChainStatus 1000b0ec     cspddk:CSPDDK.dll
 0002:000000f0       __imp_DDKSdmaClearBufDescStatus 1000b0f0     cspddk:CSPDDK.dll
 0002:000000f4       __imp_DDKSdmaInitChain     1000b0f4     cspddk:CSPDDK.dll
 0002:000000f8       __imp_DDKSdmaOpenChan      1000b0f8     cspddk:CSPDDK.dll
 0002:000000fc       __imp_DDKSdmaStopChan      1000b0fc     cspddk:CSPDDK.dll
 0002:00000100       \177CSPDDK_NULL_THUNK_DATA 1000b100     cspddk:CSPDDK.dll
 0002:00000104       __imp_I2CCloseHandle       1000b104     i2csdk:I2CSDK.dll
 0002:00000108       __imp_I2CTransfer          1000b108     i2csdk:I2CSDK.dll
 0002:0000010c       __imp_I2CSetFrequency      1000b10c     i2csdk:I2CSDK.dll
 0002:00000110       __imp_I2CSetMasterMode     1000b110     i2csdk:I2CSDK.dll
 0002:00000114       __imp_I2COpenHandle        1000b114     i2csdk:I2CSDK.dll
 0002:00000118       \177I2CSDK_NULL_THUNK_DATA 1000b118     i2csdk:I2CSDK.dll
 0002:0000011c       __imp_timeSetEvent         1000b11c     mmtimer:MMTimer.dll
 0002:00000120       __imp_timeKillEvent        1000b120     mmtimer:MMTimer.dll
 0002:00000124       \177MMTimer_NULL_THUNK_DATA 1000b124     mmtimer:MMTimer.dll
 0002:000001d8       ?szNames@?1??GetListText@MixerControlInputMux@@QAAXPAUtMIXERCONTROLDETAILS_LISTTEXT@@K@Z@4PAPBGA 1000b1d8     wavedev2_common_topaz_v1:mixerdrv.obj
 0002:000001e0       __security_cookie          1000b1e0     corelib0:seccinit.obj
 0002:000001e4       __security_cookie_complement 1000b1e4     corelib0:seccinit.obj
 0002:000001ec       ?g_BitsPerSample@@3GA      1000b1ec     wavedev2_common_topaz_v1:hwctxt.obj
 0002:000001f0       ?g_pHWContext@@3PAVHardwareContext@@A 1000b1f0     wavedev2_common_topaz_v1:hwctxt.obj
 0002:00000208       ?ms_PitchTable@CMidiStream@@0PAKA 1000b208     wavedev2_common_topaz_v1:midistrm.obj
 0002:00000238       ?ms_PitchTableInverseSampleRate@CMidiStream@@0KA 1000b238     wavedev2_common_topaz_v1:midistrm.obj
 0002:0000023c       _exitflag                  1000b23c     corelib0:cexit.obj
 0002:00000240       __onexitend                1000b240     <common>
 0002:00000244       __onexitbegin              1000b244     <common>
 0002:00000248       g_pcsExit                  1000b248     <common>
 0002:0000024c       _pRawDllMain               1000b24c     <common>

 entry point at        0001:000090f0

 Static symbols

 0001:00008ff4       _DllMainCRTStartupHelper   10009ff4 f   corelib0:pegdmain.obj
 0001:00009120       doexit                     1000a120 f   corelib0:cexit.obj
